:020000040100F9
:10000000FD6293820240FD12E39F02FE374100022F
:1000100013010100B711000293818193B71500010C
:10002000938585103716000113068613B706000264
:100030009386861539A083A2050023A0560091055A
:100040009106E3EAC5FEB70500019385850B3706E7
:10005000000113060621B70600029386060039A0A8
:1000600083A2050023A0560091059106E3EAC5FE90
:10007000B705000293858518370600021306464B24
:1000800021A023A005009105E3EDC5FEB702000203
:100090009382020C73905230B7000001E780600B2E
:1000A000B7000001E780600BB7100001E780E09324
:0800B00073005010F5BF8280BF
:1000B8000000000000000000000000000000000038
:1000C8000000000000000000000000000000000028
:1000D8000000000000000000000000000000000018
:1000E8000000000000000000000000000000000008
:1000F80000000000000000000000000000000000F8
:1001080000000000000000000000000000000000E7
:1001180000000000000000000000000000000000D7
:1001280000000000000000000000000000000000C7
:1001380000000000000000000000000000000000B7
:1001480000000000000000000000000000000000A7
:100158000000000000000000000000000000000097
:100168000000000000000000000000000000000087
:100178006F004000130141F806C00AC20EC412C63F
:1001880016C81ACA1ECC22CE26D02AD22ED432D6CF
:1001980036D83ADA3EDC42DEC6C0CAC2CEC4D2C6BF
:1001A800D6C8DACADECCE2CEE6D0EAD2EED4F2D6AF
:1001B800F6D8FADAFEDC97000000938000058290FA
:1001C80082401241A2413242C2425243E243724447
:1001D80082541255A2553256C2565257E257725897
:1001E80086481649A649364AC64A564BE64B764CC7
:1001F800865C165DA65D365EC65E565FE65F1301D9
:08020800C1077300203001A0C2
:100210003D432A876373C3029377F700BDEFADE5D3
:10022000937606FF3D8ABA960CC34CC30CC74CC7E5
:100230004107E36BD7FE11E28280B306C3408A0612
:100240009702000096966780A6002307B700A306D2
:10025000B7002306B700A305B7002305B700A30422
:10026000B7002304B700A303B7002303B700A3021A
:10027000B7002302B700A301B7002301B700A30012
:10028000B7002300B700828093F5F50F93968500A1
:10029000D58D93960501D58D61B79396270097026A
:1002A000000096968682E78086FA9680C1171D8F99
:1002B0003E96E374C3F8A5B7B70705000947D8CF42
:1002C000B7170500938707C0984385669386064055
:1002D000558F98C398471367074098C7B71708000A
:1002E0009387074023A0070023A2070023A4070049
:1002F0001307A008D8C77D57D8CF354798C3D84F24
:10030000935657018D8AE5DE8280B71708009387E0
:10031000074023A0070023A2070023A4070023A669
:1003200007007D57D8CF23A40702B717050093878E
:1003300007C09843F1769386F63F758F98C3984728
:100340001377F7BF98C7B7070500094798D382808E
:10035000B71708009387074088D7D84F137707044B
:100360006DDF828003A3418637150800B7450F0073
:1003700023A4018681470146130505409385152472
:100380000328C501B308F30013780802630A0802C2
:1003900011CE23A2118737470F0023A4F18613073C
:1003A00007246395E70005472387E184B717080012
:1003B00093870740C8534205418182800546C9B7EB
:1003C0008507E39DB7FE7DD2B7470F0093870724CB
:1003D00023A4F18623A21187F9B7411106C622C4CE
:1003E00026C2AA84EF007028E1689388086A014851
:1003F0008147014781460146B70520C726853794C6
:100400009800EF00F00B130414687D1419E40D45F7
:10041000B240224492444101828085452685EF0006
:10042000302605897DF10145E5B7411122C4130647
:1004300000109305F00F1385C18606C6D13B83A536
:1004400081849386C1861306001013850182EF0014
:1004500090341384C186814793050410130600105D
:10046000B306F4003387F50083C606000347070090
:10047000639AE6008507E395C7FE0545B24022442E
:10048000410182800145DDBF411126C293878184ED
:100490008C43B70700804AC0BE9523AEB18406C620
:1004A00022C4939745019384818489E7138501824F
:1004B000EF00302A8C409386C18613850182938693
:1004C000061013060010EF00102485371384C18630
:1004D00011E989472383F400B2402244924402493F
:1004E000410182809C4083D68185938707109CC000
:1004F00013060010B68763F4C600930700109387B5
:1005000007F01306100F9305F00F1305F410239C4A
:10051000F18413040420ED39A2853D461385C1966C
:10052000EF00D02822852244B240924402493D4641
:100530009305F00F4101E9B95D7113068002814511
:10054000280886C6F131BD47230CF1008947230EE8
:10055000F1003ED2E177938707082C080A85231A19
:10056000F102DD23B640616182805D71A2C4138512
:10057000018286C6A6C2CAC0EF00E06A1385018266
:10058000EF00C07D854513850182EF00700F8D4718
:10059000814463E3A700AA84894513850182EF00A3
:1005A000300E937725002A8689E713662500137697
:1005B000F60F9377060499C31376F60BA685138579
:1005C0000182EF00500FE1689388086A0148814773
:1005D000014781460146B705203813850182EF00A7
:1005E000206EE16838009388086A13080002854687
:1005F00081470146B70599EB138501822304010069
:10060000EF00006CB715000151469385450F680057
:10061000EF00D01913890182832709006C0051462D
:100620003ED085473ED26810C1673ED4EF00101817
:10063000B70607009C423707F1FF7D17F98F0810B6
:100640009CC22525B64026449644064961618280B5
:10065000411106C65D39113FB707008073905730CE
:10066000B70000808290B24041018280411122C4D3
:1006700006C69387818483C7670085461384818477
:10068000638ED70009476388E70023030400B24064
:100690002244410182801305000F5D39B71708001D
:1006A00093870740D84F218B09C7D84F136787001E
:1006B000D8CF793FD9BF411106C622C426C24AC04D
:1006C0008347350005476389E70611472A84638914
:1006D000E7009DC7B2402244924402494101828012
:1006E00083D7818591C34D3383474400034754002A
:1006F000E2074207BA9723A0F18623A4F184D9BF69
:1007000083D48185034604001385C19626959305FD
:100710004400EF00B00983470400BE94C204C180C6
:10072000239C91849307F00FE3F697FA2244B2409A
:1007300092440249410189BB3D45193983D78185DE
:1007400099E72244B24092440249410111B72D3B3E
:1007500083C7E184FDD7BDBF41119386818403DF48
:10076000460026C483A2818622C637150800B748F2
:100770000F0037430F004AC2814723AA018413099F
:10078000FFFF814E81468145814301480146138721
:100790008184130505409388182413030324138EC2
:1007A000C1A7636BE60363850E0009462303C700F8
:1007B00099C2A388F18499C123AA718463040800B3
:1007C00023A4518683476700A9E33244A244124917
:1007D0001385C1A74101C5B581420328C50113781E
:1007E0000802631908028502E39912FF99C2A388DF
:1007F000F18499C123AA7184B7470F009387072416
:1008000023A4F18685472303F7003244A24412490A
:1008100041018280E38C62FC03284502937FF80F3C
:10082000637D26011378F80FC29385453308CE0007
:100830002300F80105060548ADB7B307704093F7EC
:10084000F70F6394FF008546D5B7854EEDBF0111C4
:1008500026CA4EC652C4B7490F00371ADCBA22CC9A
:100860004AC856C25AC006CE938481849389F9231C
:10087000930A0006130B0009391AED3483A7418649
:10088000A383A40063F3F900E13383C7640099C331
:10089000F13BE5B783C67400638356096388660538
:1008A000930700036381F60603C701858D47998F7F
:1008B0008E07B357FA0093F7F70F639FF606930777
:1008C000170093F7F70F2388F1841147639DE70022
:1008D0003D45BD3C13850182093629CD1305000F26
:1008E000853C2388018423A2018641BF3D4523A284
:1008F000018623880184A93C0145993C0945893C2E
:100900000145B9349DBF3D4523A20186238801845A
:100910008134893C05052392A4003D45DDB73D4562
:1009200023A201862388018425343D3583C76400D2
:10093000A5F3E5B73D456DB7238801843DBF01119F
:1009400006CE22CCD53E13850182F12C138501827F
:100950003121E1689388086A01488147780085461B
:100960000146B705D9EB1385018223060100892EC4
:10097000E1689388086A014881470147814601463A
:10098000B70538FF13850182252EEFF0FF92C135A0
:100990000547AA876305E50209476300E5060545A3
:1009A00091EBB7060600DC4A7D771307F73FF98F16
:1009B000DCCA014582807D1719EB0D4582809306C4
:1009C000004037A7070013070712B7050500905D21
:1009D0007D8E75D2370606005C4A7D771307F73F98
:1009E000F98FD58F41115CCA02C613073006B24792
:1009F0006359F70001454101828085669386068030
:100A0000C9B7B24785073EC6DDB791476307F50210
:100A100063EAA7008547630AF50489476309F5047B
:100A200005458280A147E31DF5FE0947094501A858
:100A3000FD1781EFC8D20D45828005470D45B7A748
:100A4000070093870712B7060500905E798E6DD276
:100A50008A05C98D4111CCD202C613073006B247B0
:100A6000635AF7000145410182801147C9BF214700
:100A70000145F1B7B24785073EC6D5B70547AA87F6
:100A80006305E50209476304E506054591EBB706F2
:100A900006009C4A7D771307F73FF98F9CCA0145F2
:100AA00082807D1719EB0D4582809306004037A7A1
:100AB000070013070712B7050500905D7D8E75D2FC
:100AC000370706001C4B7D761306F63FF18FD58F56
:100AD0001CCB232C070085471CCF411102C61307EE
:100AE0003006B2476359F7000145410182808566AF
:100AF000938606806DBFB24785073EC6DDB711C934
:100B00008547630DF50205458280FD1791EB0D4584
:100B100082800946B7A7070093870712B70605002A
:100B2000985E718F7DD34111C8D602C61307300677
:100B3000B2476357F7000145410182800546D9BF9E
:100B4000B24785073EC6EDB7011126CAB7040600B5
:100B5000DC4806CE22CC4AC84EC652C456C2F19BCF
:100B6000DCC89C482A89C845F19B9CC8D84883C7E3
:100B7000C5012E84137737C08A07D98FDCC883C795
:100B8000D50198489A071377F7C393F7073CD98F95
:100B90009CC8FD3B0C44AA8A03454400BD35184857
:100BA000B70705002A8A98C358480850D8C3184C7C
:100BB00098C7E935AA8948509937834704002A879E
:100BC00093F6170089E6D44893E62600D4C893F636
:100BD000270099E637060600544A93E6160054CAE1
:100BE00093F6470099E637060600144A93E6260076
:100BF00014CAA18B99E7B70606009C4A93E7170031
:100C00009CCAF24062442320590123224901232433
:100C100039012326E900D244B249224A924A4A8540
:100C2000424905618280011106CE22CC02C402C66F
:100C30002147B707050037550800D8C705448D4739
:100C40008A85130505803EC022C2292A375508002F
:100C50009307C0038A851305058022C222C43EC0C3
:100C60001122F240624405618280411122C406C60D
:100C70002A84553F18405C4F93E707015CCF1C4422
:100C80001CCB5C4085CB1C43B7061000D58F1CC322
:100C9000144C5C48B240D606CE07D58F834604017B
:100CA000C206D58F8346C4012244E206D58F1CCFED
:100CB000410182801C43B706F0FFFD16F58FC1BFCE
:100CC000032305002A8E0325C30113650502232E85
:100CD000A3002324C3001396260149824D8E2326A8
:100CE00003012322C300139605016354060299C22F
:100CF0000545B1CB01476346D700639C08020D450B
:100D000082803386E700034606000507230AC300F6
:100D1000DDB799C2054505CB8147E3D0D7FE032651
:100D20000E00034546013306F70085072300A600A1
:100D3000EDB783270E00FD18DC4F93F70702D5DFD0
:100D400011656D8D11E18280B707070083C74701E8
:100D500013F585001D8D3335A00082801C4141476D
:100D6000D8CF8280B7470800938707402A8863045A
:100D7000F508B7570800938707806304F50A3747DB
:100D80000800630DE50A05458280331E1F01337696
:100D9000DE0129C683A345008843139318003396C8
:100DA0006F001346F6FF13F43300718D33146400A3
:100DB000418D88C3638B5302638C0302084303AEE7
:100DC000C500718D331E6E003365C50108C38842AE
:100DD000698E884533156500498E90C2850833D5E4
:100DE0001E0145F53244410182802326C801F9B72E
:100DF0002324C801E1B7B716050037170500B71758
:100E00000500938646C1130707C19387C7C083AE09
:100E100005008148054F8D4F914233D51E0105EDE8
:100E20008280B716050037170500B71705009386AF
:100E300006C21307C7C1938787C1D1BFB716050084
:100E400037170500B7170500938686C0130747C0FC
:100E5000938707C06DBF331E1F013376DE0119E291
:100E6000850865BF411122C635B7E1689388086AD5
:100E700001488147014781460146B705200689B5EB
:100E8000011106CEA307010089476393F502B70558
:100E90002035E1681307F1009388086A014881470B
:100EA00085460146313DF2400345F10005618280EF
:100EB000B7052005F9BF011106CE22CC26CA2306AC
:100EC000B100AA84A306C1004D37E1689388086A7F
:100ED00001487C00014789460146B78520012685E7
:100EE0000964F93B130414717D1419E40D45F240B3
:100EF0006244D24405618280854526855137058943
:100F000065F50145EDB7011106CE22CC26CA2E8427
:100F10004AC8AA84328936C6893FB247E168228628
:100F20009388086A01480147CA86B78580022685EA
:100F3000616479331304146A7D1411C485452685D0
:100F40008137058975F9F2406244D244424905610E
:100F50008280011106CE22CC26CA2EC6AA84313741
:100F60003246E1689388086A014881470147814613
:100F7000B705802026856164A1331304146A7D14AB
:100F800011C485452685ED3D058975F9F240624419
:100F9000D24405618280E16836879388086AB28608
:100FA00001482E868147B705800319BBB3C7A5004A
:100FB0008D8BB308C500B1E78D4763F4C704937701
:100FC00035002A87B9EB13F6C8FFB306E64093074E
:100FD000000263C8D706AE86BA876371C70203A84A
:100FE00006009107910623AE07FFE3EAC7FE9307C9
:100FF000F6FF998FF19B91073E97BE9563661701A7
:1010000082802A87637E150383C70500050785054F
:10101000A30FF7FEE39AE8FE828083C6050005076A
:1010200093773700A30FD7FE8505D1DF83C6050070
:10103000050793773700A30FD7FE8505F9FF61B742
:101040008280411122C61304000283A3050083A2FB
:10105000450083AF850003AFC50083AE050103AE35
:10106000450103A3850103A8C50194511307470255
:10107000B307E640232E77FC232057FE2322F7FFF9
:101080002324E7FF2326D7FF2328C7FF232A67FE51
:10109000232C07FF232ED7FE93854502E347F4FA5E
:1010A000AE86BA876371C70203A80600910791064E
:1010B00023AE07FFE3EAC7FE9307F6FF998FF19B84
:1010C00091073E97BE9563651701324441018280C6
:1010D00083C7050005078505A30FF7FEE387E8FE34
:1010E00083C7050005078505A30FF7FEE392E8FE19
:1010F000E9BF000020000000010000000300000024
:0811000006000000EB000000F6
:1011080000000700000000000000000000000000D0
:1011180000000000000000000000000000000000C7
:081128000000000000000000BF
:08113000000000800000000037
:0400000501000000F6
:00000001FF
